:020000040000FA
:06000000CDEF12F012002A
:06080000CDEF12F0120022
:060808000BEF10F01200DE
:0608180056EF10F0120083
:06082A000100CE250000D4
:08083000FE00000002000000C0
:08083800D9CFE6FFE1CFD9FFA3
:10084000E652A09A6A6A686A706A020EE66EE66A02
:10085000E66A710EE66E0F0EE66EA3EC12F00B6EFA
:10086000050EE15E0B50160E6F6E9F0E6B6E7B0ECB
:10087000696EDF6ADF500B6E0C6A0C0E0B5C000EAB
:100880000C5810E2DF50040DF3CFE9FFF4CFEAFF7C
:10089000000EE926040EEA22EE6AEE6AEE6AEE6ABD
:1008A000DF2AE8D76D8C6E6A6D986D9C68A607D0BC
:1008B00068960101186B1D6B1E6B1F6BF7D701014A
:1008C000010E316F326F336B346B256BDF6A030EB1
:1008D000DF5C26E2EA6ADF34FE0BEA36E96E0E0ED2
:1008E000E926010EEA22EE6AED6AEA6ADF34FE0BBF
:1008F000EA36E96E080EE926010EEA22EE6AED6A92
:10090000DF50EA6A290FE96E010EEA22EF6ADF5032
:10091000EA6A2C0FE96E010EEA22EF6ADF2AD7D7C6
:100920000101080E0E6F040E0F6F160E706E04019B
:10093000300E026F040E036F080E016F840E006FFD
:100940000101016B006BE552E552E7CFD9FF1200C0
:10095000D9CFE6FFE1CFD9FFE6520101000507E15B
:100960006DBA05D0686A69806988020E006F6850A8
:10097000040B06E06950040B03E06894B9EC0AF03C
:100980006DA202D0A19A97D06850010B09E069507E
:10099000010B06E051DFA08A0101040E006F689090
:1009A0006850100B06E06950100B03E0A4EC0AF04D
:1009B000689868AC19D069AC0FD0010EE66EE66A93
:1009C000000EE66EE66A730EE66EE66AA0EC11F0C3
:1009D0000B6E060EE15E0B50689C01012F5101E089
:1009E0002F072F5101E10BDA6850200B05E0695009
:1009F000200B02E08BEC0AF06850020B13E0695008
:100A0000020B10E0010EE66EE66A000EE66EE66A84
:100A1000E6687F0EE66EA0EC11F00B6E060EE15E4E
:100A20000B506A6A040E0101E76E0019E8AE02D0AD
:100A3000E73402D0E750005D02E2A19A3CD069A6FB
:100A400039D0DF6A040EDF5C35E268A632D06CCFA5
:100A500026F101012651780BE842E842E842276F6F
:100A6000689626B508D02751EA6A2C0FE96E010E68
:100A7000EA22EF7007D02751EA6A290FE96E010ECA
:100A8000EA22EF70275103E1D0EC0AF010D0000EFB
:100A9000E66EE66A260EE66E010EE66E720EE66EF3
:100AA000E66AA0EC11F00B6E060EE15E0B50DF2A39
:100AB000C9D700D0A19AE552E552E7CFD9FF12007D
:100AC000D9CFE6FFE1CFD9FF020EE126FD0EDBA470
:100AD00007D0E66AFE0EDBCFE6FF22DAE552E552EA
:100AE000FD0EDBA208D0010EE66EFE0EDBCFE6FFA8
:100AF00017DAE552E552FE0EDB500C6A700F0B6EF2
:100B00000F0E0C220BC0DEFF0CC0DDFFDECFE9FFB5
:100B1000DDCFEAFFFD0EDBCFEFFF020EE15C02E26C
:100B2000E16AE552E16EE552E7CFD9FF1200D9CF75
:100B3000E6FFE1CFD9FF020EE126FD0EDB500FE00C
:100B4000FE0EEA6ADB34FE0BEA36E96E0E0EE9268B
:100B5000010EEA22EECFDEFFEDCFDDFF0ED0FE0E5E
:100B6000EA6ADB34FE0BEA36E96E080EE926010E6E
:100B7000EA22EECFDEFFEDCFDDFFD9CFE9FFDACFFE
:100B8000EAFFEE50ED1003E1F36AF46A49D0DECFDC
:100B9000E9FFDDCFEAFF020EE926000EEA22FB0E96
:100BA000DBCFEEFFFC0EDBCFEDFFDECFE9FFDDCFCD
:100BB000EAFFEE52FA0EDBCFEFFF400E0B6EDECFF8
:100BC000E9FFDDCFEAFF0B50EF16880E0B6EDECF8C
:100BD000E9FFDDCFEAFF0B50EF12FD0EDB500CE01A
:100BE000FE0EEA6ADB34FE0BEA36E96E0E0EE926EB
:100BF000010EEA22EF740BD0FE0EEA6ADB34FE0B24
:100C0000EA36E96E080EE926010EEA22EF74DECF1D
:100C10000BF0DDCF0CF00BC0F3FF0CC0F4FF00D0E5
:100C2000020EE15C02E2E16AE552E16EE552E7CFD5
:100C3000D9FF1200D9CFE6FFE1CFD9FF020EE1269E
:100C4000FE0EDB5020E106C1E9FF07C1EAFFEE52CC
:100C5000080EEF6E06C1E9FF07C1EAFF020EE926A2
:100C6000000EEA22300EEE6E040EED6E06C1E9FFB4
:100C700007C1EAFF8C0EEF6E0EC1E9FF0FC1EAFF5C
:100C8000840EEF6E3DD0FD0EDB50E8240D6EFE0E9F
:100C9000DB50040DF3500D24040DF3CF0BF0F4CF13
:100CA0000CF0000E0B26040E0C220BC0DEFF0CC055
:100CB000DDFF840E0B6EDECFE9FFDDCFEAFF0B50C8
:100CC000EF12FD0EDB50E8240D6EFE0EDB50040D1E
:100CD000F3500D24010F040DF3CF0BF0F4CF0CF003
:100CE000000E0B26040E0C220BC0DEFF0CC0DDFF35
:100CF000840E0B6EDECFE9FFDDCFEAFF0B50EF1263
:100D0000020EE15C02E2E16AE552E16EE552E7CFF4
:100D1000D9FF1200D9CFE6FFE1CFD9FF6DA84ED0A1
:100D2000FE0EEA6ADB34FE0BEA36E96E0E0EE926A9
:100D3000010EEA22EE50EFCFEAFFE96E400EEE160A
:100D4000EE6AEE6AEE6AFE0EEA6ADB34FE0BEA3603
:100D5000E96E0E0EE926010EEA22EE50EFCFEAFF11
:100D6000E96EEE7CFE0EEA6ADB34FE0BEA36E96ED3
:100D70000E0EE926010EEA22EF74400E0B6EFE0EF7
:100D8000EA6ADB34FE0BEA36E96E0E0EE926010E46
:100D9000EA22EE50EFCFEAFFE96E0B50EF16FE0E9F
:100DA000EA6ADB34FE0BEA36E96E0E0EE926010E26
:100DB000EA22EE50EFCFEAFFE96EEF7CE552E7CF93
:100DC000D9FF12006D6A696A0101006B00D0120040
:100DD0000101005113E16D6A696A160E6F6E9F0E74
:100DE0006B6E7B0E696ED08EA28AA08AF28E6DB673
:100DF00002D06D86FCD70101010E006F12000101C7
:100E000031514DE1010E316F325149E1010E326F26
:100E1000020E155D0DE10EC1E9FF0FC1EAFFEE52B2
:100E2000EF6A0EC1E9FF0FC1EAFFC80EEF6E37D0BF
:100E3000150535E1286B04C1E9FF05C1EAFFEE5253
:100E4000080EEF6E04C1E9FF05C1EAFF020EE926B4
:100E5000000EEA22300EEE6E040EED6E04C1E9FFC4
:100E600005C1EAFF840EEF6E010E286F06C1E9FF8F
:100E700007C1EAFFEE52080EEF6E06C1E9FF07C197
:100E8000EAFF020EE926000EEA22300EEE6E040E94
:100E9000ED6E06C1E9FF07C1EAFF800EEF6E12009A
:100EA0000101336B346B020E155D1AE106C1E9FFD7
:100EB00007C1EAFFEE52080EEF6E06C1E9FF07C157
:100EC000EAFF020EE926000EEA22380EEE6E040E4C
:100ED000ED6E06C1E9FF07C1EAFFC80EEF6E1FD035
:100EE00019510401365D01011A510401375904E218
:100EF00036C419F137C41AF1D1D80EC1E9FF0FC1B8
:100F0000EAFF020EE926000EEA22380EEE6E040E0B
:100F1000ED6E0EC1E9FF0FC1EAFFC80EEF6E1200C1
:100F2000D9CFE6FFE1CFD9FF020EE126000EDE6E3B
:100F3000040EDD6EFD0EDB50E8240D6EFE0EDB5060
:100F4000040DF3500D24040DF3CF0BF0F4CF0CF08F
:100F5000D9CFE9FFDACFEAFF0B50EE260C50ED2295
:100F6000DECFE9FFDDCFEAFFEF9EFD0EDB500FE1A4
:100F7000FE0EEA6ADB34FE0BEA36E96E080EE9265D
:100F8000010EEA22DECFEEFFDDCFEDFF0ED0FE0E2A
:100F9000EA6ADB34FE0BEA36E96E0E0EE926010E34
:100FA000EA22DECFEEFFDDCFEDFFDECFE9FFDDCFC2
:100FB000EAFFEF9CDECFE9FFDDCFEAFF040EE92672
:100FC000000EEA22EF8C020EE15C02E2E16AE552D9
:100FD000E16EE552E7CFD9FF12006D98010118BF0D
:100FE0002BD01DAF09D0020E156F345101E158DF2F
:100FF0000101326B316B1FD006C1E9FF07C1EAFF67
:10100000EE52080EEF6E06C1E9FF07C1EAFF020EBD
:10101000E926000EEA22300EEE6E040EED6E06C1D9
:10102000E9FF07C1EAFF8C0EEF6E0EC1E9FF0FC1A9
:10103000EAFF840EEF6E31D0040130AF0DD0010114
:10104000010E156F335101E12BDF0101326B316B62
:10105000305101E1D4DE21D00101020E156F06C12D
:10106000E9FF07C1EAFFEE52080EEF6E06C1E9FF85
:1010700007C1EAFF020EE926000EEA22300EEE6EEC
:10108000040EED6E06C1E9FF07C1EAFF840EEF6EA4
:10109000326B316B305101E1B2DE1200D9CFE6FF85
:1010A000E1CFD9FFE652080EDF6E0101195D000E97
:1010B0001A590BE219C1DFFF145103E1010E146F3D
:1010C00004D0140502E1020E146FDF500B6E0C6A9F
:1010D0000B50195D196F0C501A591A6F0EC1E9FFA8
:1010E0000FC1EAFFEE52DFCFEFFF380E226F040E82
:1010F000236F18B119D0DF5016E016C1F6FF17C1E3
:10110000F7FF162B000E17230800F550E66E22C1DC
:10111000E9FF23C1EAFF222B000E2323E552E7500B
:10112000EF6EDF06E8D717D0DF5015E016C1E9FFF4
:1011300017C1EAFF162B000E1723EF50E66E22C1EF
:10114000E9FF23C1EAFF222B000E2323E552E750DB
:10115000EF6EDF06E9D7E552E552E7CFD9FF12007F
:10116000D9CFE6FFE1CFD9FF020EE12604C1E9FFA6
:1011700005C1EAFFEE52EFCFDFFFDFCF0BF00B50E0
:1011800001011E5D000E1F5902E21EC1DFFFDF508C
:101190000B6E0C6A0B501E5D1E6F0C501F591F6F9B
:1011A000010EDB6ADF50F36E010EDBCFF4FFF3506C
:1011B000F45C16E2010EDB50EA6A380FE96E040EA9
:1011C000EA22EF50E66E1BC1E9FF1CC1EAFF1B2BB0
:1011D000000E1C23E552E750EF6E010EDB2AE2D72A
:1011E000000ED8801E55000E1F5528E206C1E9FFEB
:1011F00007C1EAFFEE52080EEF6E06C1E9FF07C114
:10120000EAFF020EE926000EEA22380EEE6E040E08
:10121000ED6E04C1E9FF05C1EAFFEF50400B07E1A5
:1012200006C1E9FF07C1EAFFC80EEF6E06D006C18E
:10123000E9FF07C1EAFF880EEF6E28D006C1E9FF7B
:1012400007C1EAFFEE52080EEF6E06C1E9FF07C1C3
:10125000EAFF020EE926000EEA22300EEE6E040EC0
:10126000ED6E06C1E9FF07C1EAFF840EEF6E205163
:10127000211107E005D021C1FAFF01012051F96ECB
:10128000FADF01011D9F305101E1B9DD020EE15C81
:1012900002E2E16AE552E16EE552E7CFD9FF1200C2
:1012A000D9CFE6FFE1CFD9FFE6520101188F020E38
:1012B000E66EE66AE66A710EE66E0F0EE66EA3EC67
:1012C00012F00B6E050EE15E0B50300EE66EE66A14
:1012D000E66A000EE66E040EE66EA3EC12F00B6EEC
:1012E000050EE15E0B506D8CDF6A030EDF5C10E2D1
:1012F000DF50EA6A290FE96E010EEA22EF6ADF5039
:10130000EA6A2C0FE96E010EEA22EF6ADF2AEDD7B6
:10131000020EE66EE66AE66A020EE66E010EE66E02
:10132000A3EC12F00B6E050EE15E0B506D9C0101FB
:10133000080E0E6F040E0F6F000E046F040E056F83
:1013400004C106F105C107F132C401F1015103E105
:10135000100E006F13D0010EE66EE66A010EE66E07
:10136000010EE66E010EE66EE66AA0EC11F00B6E61
:10137000060EE15E0B500101200E006FE552E552B2
:10138000E7CFD9FF1200800E0401305D5BE101015F
:10139000C00E186F04013351030A34E0010A0EE055
:1013A000030A03E00101186B4DD00101DE0E166F38
:1013B000230E176F120E196F1A6B44D03251F66E4E
:1013C000F76AD890F636F7369F0EF626240EF722E7
:1013D0000900F5CF16F10A00F5CF17F1020E010151
:1013E000F76A1625F66E1751F7220800F5CF19F1A6
:1013F000030EF76A1625F66E1751F7220800F5CF8F
:101400001AF120D0030E325D1AE23251F66EF76AFD
:10141000D890F636F736A10EF626240EF7220900EC
:10142000F5CF16F10A00F5CF17F116C1F6FF17C177
:10143000F7FF0800F5500101196F1A6B02D0010186
:10144000186B00D01200D9CFE6FFE1CFD9FF020E12
:10145000E1260401386B396B30511F0B020A12E090
:10146000030A0DE0010A01E042D00101188F0401D6
:1014700038810101240502E10401388338D00101DB
:10148000188F35D00101188F040134BF10D03451AA
:101490000F0BE96EEA6AD890E936EA36080EE926BB
:1014A000010EEA22EECFDEFFEDCFDDFF0FD034518B
:1014B0000F0BE96EEA6AD890E936EA360E0EE92695
:1014C000010EEA22EECFDEFFEDCFDDFFDECFE9FF3A
:1014D000DDCFEAFFEF50800B09E0DECFE9FFDDCF83
:1014E000EAFFEF50040B02E0010E386F00D001015B
:1014F00018AF07D0380E166F040E176F1881020E42
:10150000196F020EE15C02E2E16AE552E16EE5521A
:10151000E7CFD9FF120070A015D004C1E9FF05C1C3
:10152000EAFFEF5080080DE10EC1E9FF0FC1EAFFAD
:10153000EF50840806E104C1E9FF05C1EAFF8C0E03
:10154000EF6E7090689A1200698468986D8201014C
:10155000010E256F000EE66EE66AE66EE66A750E0F
:10156000E66EE66AA0EC11F00B6E060EE15E0B5023
:1015700012000101256B000EE66EE66AE66EE66A71
:10158000740EE66EE66AA0EC11F00B6E060EE15EDC
:101590000B506D92699468A402D06894FCD7120035
:1015A000D9CFE6FFE1CFD9FFE65201012D0E2F6F13
:1015B000FD0E261553E17E0E2615E8407F0B040D27
:1015C000F3CF04F1F4CF05F1000E0427040E052338
:1015D00004C106F105C107F1067504C1E9FF05C1A3
:1015E000EAFFEF503C0BE842E8420D0835E1DF6AC4
:1015F000080EDF5C23E204C1E9FF05C1EAFF020E29
:10160000E926000EEA22EE50EFCFEAFFE96EEF5036
:10161000E66EDF50EA6A300FE96E040EEA22E55208
:10162000E750EF6E04C1E9FF05C1EAFF020EE926AB
:10163000000EEA22EE2AEF22DF2ADAD704C1E9FF00
:1016400005C1EAFF020EE926000EEA22300EEE6E18
:10165000040EED6E0DD801D03AD805D0FD0E26153A
:10166000040801E159D8E552E552E7CFD9FF12004D
:101670000101146B306B336B346B286B156B0EC12F
:10168000E9FF0FC1EAFFEF9E0E750EC1E9FF0FC122
:10169000EAFFEF9E0E7506C1E9FF07C1EAFFEF9E64
:1016A000186B196B1A6B1D6B1E6B1F6B8FD8000E9E
:1016B000E66EE66AE66EE66A030EE66EE66AA0ECA1
:1016C00011F00B6E060EE15E0B50EDEF07F0020E0F
:1016D0000101155D02E144DD1ED0156B28511AE1B0
:1016E00006C1E9FF07C1EAFFEE52080EEF6E06C120
:1016F000E9FF07C1EAFF020EE926000EEA22300EDA
:10170000EE6E040EED6E06C1E9FF07C1EAFF8C0E16
:10171000EF6E01D0286B1200D9CFE6FFE1CFD9FFE1
:10172000E6520EC1E9FF0FC1EAFFEF50400B01E0A6
:10173000010EDF6E01010E75080E005D09E132C475
:101740006EFF6E5003E0100E006F02D0040E006FAB
:10175000150528E10EC1E9FF0FC1EAFF020EE926D7
:10176000000EEA22380EEE6E040EED6E97DC020ECD
:101770000101145D07E10EC1E9FF0FC1EAFF840E0C
:10178000EF6E0FD0DF5007E10EC1E9FF0FC1EAFF96
:10179000C80EEF6E06D00EC1E9FF0FC1EAFF880E3A
:1017A000EF6E0FD01DAF0CD02051211107E005D0F6
:1017B00021C1FAFF01012051F96EFADF01011D9FDD
:1017C000156BE552E552E7CFD9FF12000401305105
:1017D000600BE842E842E842E842E842000901E0E2
:1017E00058D031510C0A54E00B0A43E00C0A35E0A2
:1017F000010A26E00B0A22E0020A20E0030A1CE0AC
:10180000080A10E0010A0CE00F0A08E0030A01E0F0
:101810003FD00101188F080E006F3BD0B4DD39D0E6
:101820003FDD37D00101010E166F010E176F1881D1
:10183000010E196F188F2DD006DE2BD02BD829D092
:1018400034510101166F176B020E1627010E172374
:101850001881010E196F188F1CD00101188F040117
:101860003451EA6A020FE96E010EEA2232C4EFFF38
:1018700010D0000EE66EE66AE66EE66A020EE66ECE
:10188000E66AA0EC11F00B6E060EE15E0B5001D083
:1018900000D01200D9CFE6FFE1CFD9FF050EE12637
:1018A0000401320510E130511F0B00090CE1010168
:1018B000188F030E0401315D04E10101010E246F54
:1018C00002D00101246B0401325101E020D13051DA
:1018D0001F0B020801E01BD134510F0B000901E17D
:1018E00016D134510F0B020801E211D1200E010173
:1018F000005D01E00CD1188F040134BF1AD03451BF
:101900000F0BE96EEA6AD890E936EA36080EE92646
:10191000010EEA22EECFDEFFEDCFDDFF34510F0BDB
:10192000EA6A2C0FE96E010EEA22020EEFCFDBFF0E
:1019300019D034510F0BE96EEA6AD890E936EA36CD
:101940000E0EE926010EEA22EECFDEFFEDCFDDFF1F
:1019500034510F0BEA6A290FE96E010EEA22020EDA
:10196000EFCFDBFFD950020FE96EDACFEAFFEF507D
:10197000010B03E1000EDF9401D0DF8434BF10D0EF
:1019800034510F0BE96EEA6AD890E936EA36080E50
:10199000E926010EEA22DECFEEFFDDCFEDFF0FD00C
:1019A00034510F0BE96EEA6AD890E936EA360E0E2A
:1019B000E926010EEA22DECFEEFFDDCFEDFF030EBA
:1019C000315D23E1DECFE9FFDDCFEAFFEF50800B91
:1019D00013E034BF09D034510F0BEA6A2C0FE96EC3
:1019E000010EEA22EF8208D034510F0BEA6A290F68
:1019F000E96E010EEA22EF82840E0B6EDECFE9FF64
:101A0000DDCFEAFF0B50EF1282D0DF74DECFE9FFAB
:101A1000DDCFEAFFEF50800B1BE0DECFE9FFDDCF2B
:101A2000EAFFEF9EDECFE9FFDDCFEAFFEF8C020E8B
:101A3000E66EE66ADECFE6FFDDCFE6FF050EE66E78
:101A4000E66AA0EC11F00B6E060EE15E0B5005D0BD
:101A5000DECFE9FFDDCFEAFFEF8CDF74D950020F54
:101A6000E96EDACFEAFFEF50020B07E1DECFE9FFC4
:101A7000DDCFEAFFEF50800B2DE0040134BF09D029
:101A800034510F0BEA6A2C0FE96E010EEA22EF9235
:101A900008D034510F0BEA6A290FE96E010EEA22D1
:101AA000EF923B0E0B6EDECFE9FFDDCFEAFF0B506E
:101AB000EF16020EE66EE66ADECFE6FFDDCFE6FF4A
:101AC000050EE66EE66AA0EC11F00B6E060EE15E06
:101AD0000B5008D03B0E0B6EDECFE9FFDDCFEAFFE7
:101AE0000B50EF16040134510F0B0C6A700F0B6E84
:101AF0000F0E0C22030E0BC0DBFF040E0CC0DBFF2D
:101B0000030EDBCFE9FF040EDBCFEAFFEF90050EFB
:101B1000E15C02E2E16AE552E16EE552E7CFD9FF0E
:021B20001200B1
:0E1B2200040130511F0B010801E04AD0305180
:101B3000600BE842E842E842E842E842010801E07E
:101B400040D0345103E0340501E03BD03151220A4A
:101B500033E0030A26E0010A17E0210A0EE0010A39
:101B600001E02FD00101F60E166F000E176F080E60
:101B7000196F1A6B1881188F24D00101F60E166F99
:101B8000000E176F188F1DD036C41EF137C41FF119
:101B90000101800E1B6F050E1C6F206B216B1D8FCA
:101BA00010D00101800E166F050E176F070E196F0A
:101BB0001A6BC10E186F05D032C4F1F00101188FF5
:101BC00000D012000501806B4B0E816F826B836B1E
:101BD000846B856B080E866F0001E56B1A0EE66E4E
:101BE000010EE66E60EC05F0E552E5521E0EE66E63
:101BF000020EE66E60EC05F0E552E552400EE66E30
:101C0000400EE66E050EE66EE66A020EE66E97EC94
:101C100005F00B6E050EE15E0B50F3CFEDF0F4CF47
:101C2000EEF00001EF6BF06BE66B1200D9CFE6FF30
:101C3000E1CFD9FFFD0EDBCF06F0FE0EDBCF07F0C4
:101C4000050E061801E1075002E0000E31D0FB0E30
:101C5000DBCF0BF0FC0EDBCF0CF00001ED510B18CD
:101C600002E1EE510C1813E1400EE66E400EE66EF6
:101C7000050EE66EE66A020EE66E97EC05F00B6E58
:101C8000050EE15E0B50F3CFEDF0F4CFEEF0FB0E5E
:101C9000DBCF0BF0FC0EDBCF0CF00001EF510B188B
:101CA00002E1F0510C1802E1E66BEB6B010E00D083
:101CB000E552E7CFD9FF1200D9CFE6FFE1CFD9FF38
:101CC0000001E56BED51EE1102E1000E08D0EDC010
:101CD000E9FFEEC0EAFFEF50800B01E0010E0009C2
:101CE00045E1FC0EDBCF0BF0EDC0E9FFEEC0EAFFF3
:101CF000EE52EF50D8800B5408E2EDC0E9FFEEC081
:101D0000EAFFEE52FC0EEFCFDBFFE56BFC0EDB5083
:101D1000E55D19E2E551EA6A400FE96E050EEA2237
:101D2000EF50E66EE551E76EFD0EDBCFE9FFFE0EEC
:101D3000DBCFEAFFE750E926000EEA22E552E75042
:101D4000EF6EE52BE3D7400EE66E400EE66E050E15
:101D5000E66EE66A020EE66E97EC05F00B6E050E77
:101D6000E15E0B50F3CFEDF0F4CFEEF00001E55162
:101D700000D0E552E7CFD9FF1200D9CFE6FFE1CF7F
:101D8000D9FFA09A0001E6510CE1FD0EDBCFE7F090
:101D9000FE0EDBCFE8F0FC0EDBCFEBF0010EEC6FBC
:101DA000E66FA08AE552E7CFD9FF1200D9CFE6FF50
:101DB000E1CFD9FF030EE126A09A0001E65102E02F
:101DC000A08A2FD0DF6AFD0EDBCF06F0FE0EDBCF40
:101DD00007F0DE5206C0DEFF07C0DDFFDD52DF2A5E
:101DE000DF500B6E0C6AFF0E0B1801E10C5001E185
:101DF0000BD0010EDBCFE9FFDB2A020EDBCFEAFFBF
:101E000001E3DB2AEF50EBE1FD0EDBCFE7F0FE0E46
:101E1000DBCFE8F0DFCFEBF00001010EEC6FE66FF7
:101E2000A08A030EE15C02E2E16AE552E16EE5524E
:101E3000E7CFD9FF1200D9CFE6FFE1CFD9FF030EDC
:101E4000E126A09A0001E65102E0A08A30D0DF6AC4
:101E5000FD0EDBCF06F0FE0EDBCF07F0DE5206C034
:101E6000DEFF07C0DDFFDD52DF2ADF500B6E0C6A9C
:101E7000FF0E0B1801E10C5001E10CD0010EDBCF7D
:101E8000F6FFDB2A020EDBCFF7FF01E3DB2A0800B7
:101E9000F550EAE1FD0EDBCFE7F0FE0EDBCFE8F018
:101EA000DFCFEBF00001EC6B010EE66FA08A030EB2
:101EB000E15C02E2E16AE552E16EE552E7CFD9FF6B
:101EC0001200D9CFE6FFE1CFD9FF020EE126A09A9A
:101ED0000001EF51F01102E1000E08D0EFC0E9FF60
:101EE000F0C0EAFFEF50800B01E0010E000902E0B4
:101EF000A08A87D0030EE65D01E1E66BE65102E1C0
:101F0000A08A7FD0020EE65D16E1E66A000EE66E5C
:101F1000E66A010EE66E020EE66E97EC05F00B6EB9
:101F2000050EE15E0B50F3CFEFF0F4CFF0F00001BF
:101F3000030EE66F65D0E60563E1400E0B6E0C6A9A
:101F4000EB510B5C000E0C5803E2400EDF6E02D02A
:101F5000EBC0DFFFDF50EB5DEB6F000EE96F050EAE
:101F6000EA6F010EDFCFDBFFEC5117E1010EDB5012
:101F700013E0E7C0F6FFE8C0F7FF0800F550E9C03E
:101F8000E9FFEAC0EAFFEF6EE92B000EEA23E72B38
:101F9000E823010EDB06EAD715D0010EDB5012E074
:101FA000E7C0E9FFE8C0EAFFEF50E9C0E9FFEAC097
:101FB000EAFFEF6EE92B000EEA23E72BE823010E80
:101FC000DB06EBD7EB5108E1400EDF5C03E1020ECC
:101FD000E66F02D0030EE66FDFCFE6FF000EE66E7F
:101FE000050EE66E010EE66E020EE66E97EC05F04B
:101FF0000B6E050EE15E0B50F3CFEFF0F4CFF0F077
:10200000A08A020EE15C02E2E16AE552E16EE5526D
:06201000E7CFD9FF12002A
:0A201600DACFE4FFE2CFDAFFE9CFF2
:10202000E4FFEACFE4FFF6CFE4FFF7CFE4FFF5CF1C
:10203000E4FFF3CFE4FFF4CFE4FFFACFE4FF00EED8
:1020400000F00B0EE80403E3EECFE4FFFBD700EE55
:102050000BF0030EE80403E3EECFE4FFFBD7E652F8
:10206000A8EC04F0E55200EE0DF0030EE80403E3E3
:10207000E5CFEDFFFBD700EE0AF00B0EE80403E31B
:10208000E5CFEDFFFBD7E5CFFAFFE5CFF4FFE5CFD6
:10209000F3FFE5CFF5FFE5CFF7FFE5CFF6FFE5CF9F
:1020A000EAFFE5CFE9FFE5CFDAFF1100D8CFE4FF83
:1020B000E0CFE4FFE46EDACFE4FFE2CFDAFFE652EE
:1020C000E552E5CFDAFFE550E5CFE0FFE5CFD8FFF9
:1020D000100008D80101005102E1E8EC06F012D826
:1020E000F9D712000F0EC11202D81CEF04F0000144
:1020F000E26BE16B010EE06FF00E8A169316928888
:10210000928A1200D9CFE6FFE1CFD9FF020EE12675
:102110008DD8200E0101E76E0019E8AE02D0E73439
:1021200002D0E750005D03E36D50020B01E074D074
:102130000001E15111E0E0510EE10001E6510BE137
:10214000B60EE66E250EE66E1BEC0FF0E552E5527C
:102150000001010EE06F01D0E06B0001E6515AE191
:10216000400EE66EA00EE66E000EE66E5CEC0EF023
:10217000E552E552E552DF6EDF504CE0010EDB6ABE
:10218000DF50F36E010EDBCFF4FFF350F45C37E267
:10219000010EDB50EA6AA00FE96E000EEA22EF5052
:1021A0000A0A16E0070A14E0010EDB50EA6AA00FE3
:1021B000E96E000EEA22EF28E66E010EDB50EA6AB5
:1021C000600FE96E000EEA22E552E750EF6E14D080
:1021D000010EDB50EA6AA00FE96E000EEA22EF5012
:1021E000E66E010EDB50EA6A600FE96E000EEA222D
:1021F000E552E750EF6E00D0010EDB2AC1D7DFCFEA
:10220000E6FF600EE66E000EE66EBDEC0EF0E552E7
:10221000E552E55261EC0FF0020EE15C02E2E16A88
:10222000E552E16EE552E7CFD9FF12000001FE5101
:10223000FF1104E1100EFE6F270EFF6FFE07000E68
:10224000FF5B6DA20AD0FE51FF1106E18A708AA0E1
:1022500002D08A8201D08A922ED00101005103E17E
:102260008A908A9228D0000503E18A808A8223D04E
:10227000020E005D03E18A808A921DD0040E005D8B
:1022800003E18A908A8217D0100E005D07E10001F9
:10229000FE51FF1102E18A708A920DD0200E005D7E
:1022A0000AE10001FE51FF1106E18A708AA002D006
:1022B0008A9201D08A821200120012008050100B04
:1022C00001E0010E0001E15D0DE1E25102E0E207F3
:1022D00008D08050100B100A01E0010EE16F640E6F
:1022E000E26F03D0E25101E0E2071200120091EF29
:1022F0000DF01200E2EF0DF00101240520E10101D3
:1023000025051DE1A09AD9DF6D920101256B000121
:10231000100EE36F0E0EE46FE307000EE45BE35173
:10232000E411FAE16D84080EE36F070EE46FE30732
:10233000000EE45BE351E411FAE16D94A08A12000F
:10234000D9CFE6FFE1CFD9FFFD0EDBCF06F0FE0EC1
:10235000DBCF07F0050E061801E1075039E0E86809
:10236000061802E17F0E071831E0030E061801E19E
:1023700007502AE0020E061801E1075023E0010E83
:10238000061801E107501CE0740E061801E1075021
:1023900015E0750E061801E107500EE0730E0618E1
:1023A00001E1075007E0720E061801E1075001E055
:1023B00010D00FD083DF0DD07FDF0BD07EDF09D0B0
:1023C00099DF07D096DF05D092DF03D08FDF01D0F1
:0E23D00000D0010E00D0E552E7CFD9FF120079
:0223DE001201EA
:1023E000000202000008D8040A00000101020001F6
:1023F00009024300020100C0320904000001020288
:102400000100052400100104240202052406000135
:1024100005240100010705810308000209040100E9
:10242000020A0000000705020240000007058202C0
:102430004000000403090434034D00690063007286
:10244000006F0063006800690070002000540065A0
:1024500000630068006E006F006C006F0067007919
:1024600000200049006E0063002E00340343004446
:102470000043002000520053002D00320033003290
:1024800000200045006D0075006C0061007400695B
:10249000006F006E002000440065006D006F00F0CA
:0724A00023332437246B24D1
:0824A8002A0EF66E080EF76E15
:1024B000000EF86E01010900F5503A6F0900F55061
:1024C0003B6F03E13A6701D03DD00900F550356F0D
:1024D0000900F550366F0900F550376F0900090003
:1024E000F550E96E0900F550EA6E0900090009008F
:1024F000F550386F0900F550396F09000900F6CF23
:102500003CF1F7CF3DF1F8CF3EF135C1F6FF36C1D2
:10251000F7FF37C1F8FF0101385302E1395307E0F3
:102520000900F550EE6E3807F8E23907F9D73CC1DB
:10253000F6FF3DC1F7FF3EC1F8FF01013A07000E6B
:062540003B5BBFD7120057
:0A254600FE0EE3CFE9FFFF0EE3CF26
:10255000EAFFE9CFF3FFEACFF4FFFB0EE35003E11C
:10256000FC0EE35009E0FB0EE30602E2FC0EE3067C
:0A257000FD0EE350EE6EF1D71200ED
:06257A00000EF36E00EEFE
:1025800000F0080E01D81200EA6002D0EE6AFCD713
:0A259000F350E9601200EE6AFCD778
:06259A0013EE00F023EE39
:1025A00000F0F86A0A9C54EC12F0E6EC12F069ECC8
:0625B00010F0FBD7120041
:0A25B600427574746F6E2050726558
:0B25C00073736564202D2D200D0A00B0
:0225CC001200FB
:0225CE0000000B
:00000001FF
